:100000000C9435000C945D000C945D000C945D0024
:100010000C945D000C945D000C945D000C945D00EC
:100020000C945D000C945D000C945D000C945D00DC
:100030000C945D000C945D000C945D000C945D00CC
:100040000C94D5010C945D000C94A3010C947D01DB
:100050000C945D000C945D000C945D000C945D00AC
:100060000C945D000C945D00FC0211241FBECFEFC8
:10007000D8E0DEBFCDBF21E0A4E1B1E001C01D9218
:10008000AC3BB207E1F711E0A0E0B1E0EAE1F7E054
:1000900002C005900D92A431B107D9F710E0C5E375
:1000A000D0E004C02197FE010E943003C433D10781
:1000B000C9F70E941F020C948B030C940000CF928E
:1000C000DF92EF92FF920F931F93CF93DF936C0118
:1000D0007A018B01C0E0D0E0CE15DF0589F0D801B0
:1000E0006D918D01D601ED91FC910190F081E02D93
:1000F000C6010995892B11F47E0102C02196ECCF2F
:10010000C701DF91CF911F910F91FF90EF90DF908A
:10011000CF900895FC01918D828D981761F0828DAA
:10012000DF01A80FB11D5D968C91928D9F5F9F732B
:10013000928F90E008958FEF9FEF0895FC01918DCD
:10014000828D981731F0828DE80FF11D858D90E03A
:1001500008958FEF9FEF0895FC01918D228D892FD7
:1001600090E0805C9F4F821B91098F7399270895BF
:100170008DE191E00E94AC0021E0892B09F420E0A0
:10018000822F0895FC01848DDF01A80FB11DA35AB1
:10019000BF4F2C91848D90E001968F739927848FA7
:1001A000A689B7892C93A089B1898C9180648C939E
:1001B000938D848D981306C00288F389E02D808189
:1001C0008F7D80830895EF92FF920F931F93CF93BB
:1001D000DF93EC0181E0888F9B8D8C8D981305C097
:1001E000E889F989808185FD24C0F62E0B8D10E009
:1001F0000F5F1F4F0F731127E02E8C8DE8120CC07C
:100200000FB607FCFACFE889F989808185FFF5CF21
:10021000CE010E94C200F1CF8B8DFE01E80FF11DCF
:10022000E35AFF4FF0820B8FEA89FB89808180625D
:1002300007C0EE89FF896083E889F989808180643D
:10024000808381E090E0DF91CF911F910F91FF902B
:10025000EF900895CF93DF93EC01888D8823C9F048
:10026000EA89FB89808185FD05C0A889B9898C91BF
:1002700086FD0FC00FB607FCF5CF808185FFF2CF5A
:10028000A889B9898C9185FFEDCFCE010E94C2006B
:10029000E7CFDF91CF91089580E090E0892B29F09E
:1002A0000E94B80081110C94000008953FB7F894A3
:1002B0008091190190911A01A0911B01B0911C012C
:1002C00026B5A89B05C02F3F19F00196A11DB11DB1
:1002D0003FBFBA2FA92F982F8827820F911DA11DEC
:1002E000B11DBC01CD0142E0660F771F881F991F29
:1002F0004A95D1F708950E9436031F920F920FB6C8
:100300000F9211242F933F934F935F936F937F939B
:100310008F939F93AF93BF93EF93FF938DE191E002
:100320000E94C200FF91EF91BF91AF919F918F9179
:100330007F916F915F914F913F912F910F900FBEE1
:100340000F901F9018951F920F920FB60F921124C5
:100350002F938F939F93EF93FF93E0912D01F09153
:100360002E018081E0913301F091340182FD12C0B1
:100370009081809136018F5F8F73209137018217B2
:1003800051F0E0913601F0E0E35EFE4F958F8093EF
:10039000360101C08081FF91EF919F918F912F9144
:1003A0000F900FBE0F901F9018951F920F920FB6CF
:1003B0000F9211242F933F938F939F93AF93BF93EB
:1003C0008091150190911601A0911701B09118012B
:1003D0003091140123E0230F2D3720F40196A11D45
:1003E000B11D05C026E8230F0296A11DB11D209363
:1003F00014018093150190931601A0931701B093F7
:1004000018018091190190911A01A0911B01B091DE
:100410001C010196A11DB11D8093190190931A0131
:10042000A0931B01B0931C01BF91AF919F918F913D
:100430003F912F910F900FBE0F901F9018957894B9
:1004400084B5826084BD84B5816084BD85B58260D9
:1004500085BD85B5816085BD80916E00816080938A
:100460006E001092810080918100826080938100F3
:100470008091810081608093810080918000816003
:10048000809380008091B10084608093B10080915E
:10049000B00081608093B00080917A008460809386
:1004A0007A0080917A00826080937A0080917A004D
:1004B000816080937A0080917A00806880937A00CE
:1004C0001092C100E0912D01F0912E0182E0808315
:1004D000E0912901F0912A011082E0912B01F09125
:1004E0002C018FEC808310923501E0913101F09165
:1004F000320186E08083E0912F01F091300180810C
:1005000080618083E0912F01F091300180818860CB
:100510008083E0912F01F091300180818068808399
:10052000E0912F01F091300180818F7D8083CC2478
:10053000CA9493E0D92EE12CF12C8091BA018E302F
:1005400008F08E508770806480937C0080917A00E0
:10055000806480937A0080917A0086FDFCCFA09120
:10056000780080917900B0E0B82B2FEF30E00E9446
:100570002903A70196010E943B03622F8DE191E0C0
:100580000E94E3008091BA019091BB0101968330F3
:1005900091052CF49093BB018093BA0104C0109292
:1005A000BB011092BA010E9456012B013C0184E16B
:1005B000882E912CA12CB12C0E945601DC01CB017C
:1005C00084199509A609B709883E9340A105B1058C
:1005D00058F021E0821A9108A108B10888EE480E6F
:1005E00083E0581E611C711C81149104A104B104A4
:1005F00019F70E944C01A1CFEDE1F1E013821282C4
:1006000088EE93E0A0E0B0E084839583A683B7836F
:1006100088E091E09183808385EC90E095878487E2
:1006200084EC90E09787868780EC90E0918B808BBC
:1006300081EC90E0938B828B82EC90E0958B848BA5
:1006400086EC90E0978B868B118E128E138E148E13
:1006500008950E947C03B7FF0895821B930B0895B1
:10066000EE0FFF1F0590F491E02D099481E090E0DA
:10067000F8940C948B03052E97FB1EF400940E94B3
:10068000520357FD07D00E945A0307FC03D04EF4D3
:100690000C94520350954095309521953F4F4F4F04
:1006A0005F4F089590958095709561957F4F8F4F1E
:1006B0009F4F0895A1E21A2EAA1BBB1BFD010DC07E
:1006C000AA1FBB1FEE1FFF1FA217B307E407F50702
:1006D00020F0A21BB30BE40BF50B661F771F881FDE
:1006E000991F1A9469F760957095809590959B0174
:1006F000AC01BD01CF010895A29FB001B39FC0011D
:10070000A39F700D811D1124911DB29F700D811D3D
:0A0710001124911D0895F894FFCF05
:10071A000100000000000000E3005F00AC008A0056
:04072A009E002A0102
:00000001FF
